:100200004F726967696E616C2046696C653A20704F
:10021000726F6A6563742E6865780D0A4F75747025
:10022000757420446174653A20323030392F303192
:100230002F31380D0A4F75747075742046696C65DE
:100240003A20657039343331783428646267292E56
:100250006865780000000000000000000000000059
:10026000000000000000000000000000000000008E
:100270000000000000000000000000000000006F0F
:102355000D0A205B48444D492076312E33204D61CE
:10236500747269785D0D0A0D0A000D0A0D0A0048A0
:102375006172647761726520494F20696E6974697D
:10238500616C20646F6E652E2E2E2E2E2E2E2E2E17
:102395000D0A0053595354454D3A2053573120697E
:1023A500732073656C65637465640D0A0053595336
:1023B50054454D3A205357322069732073656C6537
:1023C500637465640D0A0053595354454D3A2053BF
:1023D50057332069732073656C65637465640D0AF2
:1023E5000053595354454D3A2053573420697320AF
:1023F50073656C65637465640D0A005359535445E0
:102405004D3A2052554E204B45592069732073652E
:102415006C65637465640D0A0053595354454D3A10
:1024250020506F727420537769746368696E6720F2
:1024350064657465637465642E2E2E0D0A00535908
:102445005354454D3A205357256420737769746377
:102455006820746F20506F7274202558206973208E
:102465007365740D0A00525332333220434D443A9A
:1024750020537472696E6720427566666572204FD7
:10248500766572666C6F770D0A00257320255820D6
:102495002558202558202558005357430073776346
:1024A50000525332333220434D443A2053776974F6
:1024B500636820746F2025580D0A004552524F520B
:1024C5003A20506172616D32206F766572666C6F6D
:1024D500770D0A004552524F523A20506172616D94
:1024E50031206F766572666C6F770D0A0053454C27
:1024F5000073656C00525332333220434D443A2009
:1025050053656C6563742074686520535725640DA5
:102515000A005057520070777200525332333220FE
:10252500434D443A2053656C656374207468652097
:10253500706F776572207374617475732069732089
:1025450025640D0A005253540072737400525332BD
:10255500333220434D443A2053797374656D2052CC
:07256500657365740D0A00A7
:0E3BBC0041F82B0042F81F000042F8260000DE
:1030E20090F828E0FF2421F582E434F8F583229059
:1030F200F82CE0FEA3E0FFC39404EE6480948022E7
:10310200780D7CF87D017BFF120755EF2274212F89
:10311200F58274F83EF583740AF074002FF5827418
:10312200F83EF583E4F0742E2FF58274F83EF583B1
:1031320074FFF090F82DE004F02274002FF58274F1
:10314200F83EF583E4F090F82CE0FCA3E02421F5AE
:103152008274F83CF583E022780D7CF87D017BFFD8
:10316200120755EF2290F82CE0FEA3E02421F5820D
:1031720074F83EF58322E4F0A3F090F82CF0A3F06B
:103182002290F82CE004F022780D7CF87D017BFF80
:10319200120755EF22A3F0A37401F0A322742E2F7D
:1031A200F58274F83EF5832290F82574FFF0E490DE
:1031B200F828F0C211C210C20F2278007CF87D01FB
:1031C2007B017AF879217E007F042290F82CE0FCC2
:1031D200A3E022C390F82DE0940490F82CE06480E0
:1031E20094802290F8047402F022780D7CF87D011C
:0E31F2007BFF120755EF227BFF7A2479D9224A
:100A1200E4FF1242BB7D017F407E021236A17BFFC2
:100A22007A237955123E977BFF7A23796F123E978C
:100A32007BFF7A42792DE4FF12436E7B007C007DBE
:100A4200641228DE7BFF7A007956124362E4FF12B9
:100A5200403412256C7A237974120FEE90F8041246
:100A6200317B1230F1500A12310F70F6123183804D
:100A7200F11231AAC390F827E0940A90F826E09484
:100A820000405B1231781230F1503812420BEF9075
:100A9200F82C6017E0FEA3E0FF242E1231A2E0251D
:100AA200E04401FD12319FEDF0800EE0FEA3E02450
:100AB2002E1231A2E0FF25E0F012313570C812315A
:100AC2008380C3120003EF90F8256009E0FF25E060
:100AD2004401F08005E0FF25E0F0D20F8002C20F52
:100AE20090F804E014600D14605724026003020DB4
:100AF2006C020B4D301021C2107F0112414EEF24C7
:100B0200DB7015120FB01230F1500A120F8870F616
:100B120012318380F11231E5300F2090F825E06424
:100B2200FE7018120FB01230F1500A120F8870F6D0
:100B320012318380F11231E5020D6C438701020DFF
:100B42006C300F6A90F825E0B4FE06120FF5020D24
:100B52003DE412317C1230F1505412319FE0647F37
:100B6200704190F82C12316CE024F5601514601A73
:100B720014601F2403702174212F123170740BF042
:100B82008016123167740CF0800E123167740DF00A
:100B92008006123167740AF01231CDFF12314FFD17
:100BA200122FC31231357003123183020B572010FA
:100BB20003020CB6C2107F0112414EEF1205700CF7
:100BC20096050C25060C81070C8E080CA70C0C1937
:100BD200150C01170BFE1B0BF81C0C121D0C0B2025
:100BE2000BF5230BEF240C042700000CB6120FF5B3
:100BF200020C91020C81120FE1020C91020C96027E
:100C02000CA71230E2740A80131230E2740B800CCB
:100C12001230E2740C80051230E2740DF090F82864
:100C2200E080527BFF7A247900123E971230E2E094
:100C3200FEB40A0B74212F1230E9740BF08031EEEE
:100C4200B40B0C90F828E01230E7740CF0802112FB
:100C520030E2E0FEB40C0B74212F1230E9740DF077
:100C6200800EEEB40D0A90F828E01230E7740AF014
:100C720090F828E0FF1230E7E0FD122FC380357AAA
:100C8200237998120FEE90F828F08028120FE17461
:100C920001F080207BFF7A2379CC123E9790F828CE
:100CA2007402F0800F7BFF7A2379E6123E9790F868
:100CB200287403F01231BC1208F8EF601C1231BC28
:100CC200120350E490F829F0D21190F81FF0A3F02B
:100CD2007BFF7A24791E123E9790F829E014606017
:100CE200046003020D6CC390F820E094E890F81FB2
:100CF200E0940340751231787BFF7A2479431231F4
:100D0200CDFD2401FEE43C90F835F0A3CEF0742131
:100D12002D123151FF90F837E4F0A3EFF0123E9715
:100D22001231CDFF12314FFD1232001231357003F4
:100D32001231831231D540C090F8297401F0802A13
:100D4200C390F820E094B890F81FE0940B401B1277
:100D520031781231CDFF12314FFD1232001231358E
:100D620070031231831231D540E8120FFC90F82A39
:100D7200EFF0F47003020A76E0FFA3E0FE04F074E1
:100D82000D2EF582E434F8F583EFF090F82BE0D3E2
:100D92009412400E7BFF7A24796B123E97E490F80E
:100DA2002BF090F82AE0FF640A6008EF640D6003FC
:100DB200020A76E490F82BF090F86374FFF0A374C3
:100DC20024F0748F12319774FFF07480123197748B
:100DD200F8F0A3740512319874F8F0A37407123175
:100DE2009874F8F0A3740912319874F8F0A3740B94
:100DF200F07B017AF8790D12184AE490F810F07A33
:100E020024799E12310260097A2479A21231027089
:100E1200657A2479A690F807120FBBEE9400405031
:100E2200D3EF9403EE94005047A3E0FEA3E0FFC388
:100E3200940AEE94004030D3EF940DEE94005027C4
:100E420090F805A3E0FFFD90F828F090F807A3E0E2
:100E5200FC74212D1230E9ECF074212F1230E9E0FC
:100E6200FD122FC3020A767BFF7A2479C0020F2576
:100E72001231F9020F257A2479F212315A60097A75
:100E82002479F612315A702E7A2479FA90F80512E2
:100E92000FBBEE94004019D3EF9403EE9400501070
:100EA20090F805A3E01230E7E0FD123200020A7664
:100EB2001231F9020F257A25791712318A60097ADF
:100EC20025791B12318A70617BFF7A25791F90F890
:100ED20005E0FFA3E090F835CFF0A3EFF0123E97C4
:100EE20090F805E0FAA3E0FB4A700C12374290F842
:100EF200047401F0020A76EB64014A70231240A4E2
:100F0200E412317C1230F1501112313CFD122FC328
:100F120012313570EF12318380EA1231E5020A761E
:100F22001231F9123E97020A767A25794A1231EC89
:100F3200600C7A25794E1231EC6003020A767BFF4F
:100F42007A257952123E9712256CE412317C1230C6
:100F5200F1500A12310F70F612318380F11231AA68
:100F62001237421240A4E412317C1230F1501112B5
:100F7200313CFD122FC312313570EF12318380EAFA
:100F82001231E5020A7674002FF58274F83EF58379
:100F9200E4F090F82CE0FCA3E02421F58274F83C04
:100FA200F583E0FD122FC390F82DE004F0221240E9
:100FB200A4E490F82CF0A3F0227BFFE0FFA3E090E2
:100FC200F835CFF0A3EFF0123E9790F806E024FF39
:100FD200F090F805E034FFF0E0FEA3E0FFC3227BCF
:100FE200FF7A2379B2123E9790F828227BFF123EB5
:0A0FF20097E42212374290F804221F
:10005600AE07E4FF12414EBFEB09EE7006EDB41099
:0400660002D2102290
:10422D0090F827E004F0700690F826E004F03011C5
:10423D000E90F820E004F0700690F81FE004F022D4
:102E77004552524F523A2043616E6E6F7420666915
:102E87006E6420535725640A0D0053595354454D1A
:102E97003A205357256420416464723D30782530C9
:102EA7002E325820666F756E640A0D004552524FD8
:102EB700523A2053776974636820506F72742045C3
:102EC70072726F722C20535725642025580D0A0003
:102ED7004552524F523A20557064617465205452DE
:102EE7004547204572726F722C205357256420770F
:102EF7007269746520307839300D0A004552524F97
:102F0700523A20494943206661696C65642C2073F5
:102F170074617475733D50656E64696E67200D0A40
:102F2700004552524F523A20494943206661696C25
:102F370065642C207374617475733D4E6F416374BF
:102F4700200D0A004552524F523A20494943206604
:102F570061696C65642C207374617475733D546981
:102F67006D65204F7574200D0A004552524F523A35
:102F770020494943206661696C65642C207374613C
:102F87007475733D4172626974726174696F6E4CD6
:102F97006F7373200D0A004552524F523A20494928
:102FA70043206661696C65642C2073746174757362
:0C2FB7003D307825302E3258200D0A00E5
:103DFC00F07B017AF9790C90F902E4F0A37402F0EB
:103E0C00E4A3F07D7AFF2290F90FE0FEA3E02401F9
:103E1C00FFE43E90F835F0A3EF227BFF90F94EE0E3
:103E2C002401FEE43390F835F0A3CEF022E490F9AF
:0E3E3C000CF0A32290F90C7401F0A3749022F4
:10256C00E4FB7D01FF12406E7D021227177D0112E4
:10257C0027177B017D017F04121DC07B017D027F2B
:10258C0004121DC07D207F021226EF7D407F0212B7
:10259C001DC07D807F0212271F1226DB7D087F0560
:1025AC00121DC07B027D017F05121DC07D0212260B
:1025BC00DB7D407F05121DC07D807F051226EF7DDF
:1025CC00107F05121DC07D207F0512271F1226E5E6
:1025DC007D08E4FF121DC07D011226E57D02E4FF9B
:1025EC00121DC07D401227037D80E4FF121DC07DAB
:1025FC00101227037D20E4FF121DC07B027D027F99
:10260C0006121DC07B027D047F06121DC0E4FB7DFB
:10261C00027F02121DC07D0412270D7D087F02125D
:10262C001DC07D1012270D7D087F06121DC07F0175
:10263C00124356123E40F0E490F90FF0A3F090F9DB
:10264C000FE0FEA3E0FFC39404EE940040030226C7
:10265C00DAEE703AEF14601214601E146023240337
:10266C00702C1226F7122BB080061226F7122A496C
:10267C007D807F02122A498015122727122BB080E9
:10268C0006122727122A497D807F02122BB07F0168
:10269C0012433E123DFD12273390F90BEFF07BFFF6
:1026AC0060097A2E7977123E13800E7A2E79911268
:1026BC003E13F0A3E4F0A3747AF0123E9790F91055
:1026CC00E004F0700690F90FE004F002264A227B39
:1026DC00027F05121DC07B02227B02E4FF121DC08B
:1026EC007B02227B02121DC07B02227D207F021204
:1026FC002BB07D407F02227B02E4FF121DC07B02C7
:10270C0022E4FB7F02121DC0E4FB227B017F081236
:10271C001DC0227B02121DC07D04227D207F02126F
:07272C002BB07D407F02226B
:1040A4007D047F06122BB07D027F06122A497D0211
:1040B4007F08122A497D017F08122A497D017F0465
:0F40C400122A497D027F04122A497F0A02433ED5
:103742007D047F06122A497D027F06122BB07D027C
:103752007F08122BB07D017F08122BB07D017F0400
:10376200122BB07D027F04122BB07D047F05122A3A
:10377200497D087F05122A497D017F05122A497D6C
:10378200027F05122A497D407F05122A497D807FEA
:1037920005122A497D107F05122A497D207F0512D4
:1037A2002A497D04E4FF122A497D08E4FF122A49CE
:1037B2007D01E4FF122A497D02E4FF122A497D407D
:1037C200E4FF122A497D80E4FF122A497D10E4FFBA
:0A37D200122A497D20E4FF022A4973
:1032000090F94FEDF090F94EEFF014601214601E3B
:103210001460232403702C1232B7122BB0800612D4
:1032200032B7122A497D807F02122A498015123254
:10323000C3122BB080061232C3122A497D807F024E
:10324000122BB07F0112433290F94FE024F5601148
:1032500014601C14601224037025123E3974FC8023
:1032600013123E3974FD800C123E3974FE80051233
:103270003E3974FF123DFC12273390F90BEFF090AA
:10328000F90BE060177A2E79B3123E2690F94FE0E1
:10329000FF90F837E4F0A3EFF01232CF123E401265
:1032A0003DFC12273390F90BEFF0600A7A2E79D7A4
:1032B000123E261232CF227D207F02122BB07D409B
:1032C0007F02227D207F02122BB07D407F022212DE
:0B32D0003E9790F90BE0FF123EE42255
:102FC300AC05EF14604C147003023051147003020B
:102FD3003094240360030230D87D047F05122A490C
:102FE3007D087F05122A497D017F05122A497D024A
:102FF3001230D960111460121460132403600302A9
:1030030030D87D0480437D08803F7D01803B7D0275
:1030130080377D407F05122A497D807F05122A492A
:103023007D107F05122A497D201230D9601114606A
:1030330012146013240360030230D87D40800A7D9C
:103043008080067D1080027D207F050230D57D04BF
:10305300E4FF122A497D08E4FF122A497D01E4FFB7
:10306300122A497D02E4FF122A49EC24F560101468
:1030730060131460162403705C7D04E4FF80537DA9
:1030830008E4FF804D7D01E4FF80477D02E4FF807B
:10309300417D40E4FF122A497D80E4FF122A497DE5
:1030A30010E4FF122A497D20E4FF122A49EC24F59B
:1030B3006010146013146016240370197D40E4FF3C
:1030C30080107D80E4FF800A7D10E4FF80047D2072
:0F30D300E4FF122BB0227F05122A49EC24F522CC
:10420B00EF14600E14600F146010240370137D0202
:10421B00800A7D0480067D0880027D107F021237A4
:02422B00DC2293
:080003007D087F061237DC22A4
:103EE40090F956EFF024FE601214601714601C243D
:103EF4000370207BFF7A2F7903802B7BFF7A2F7945
:103F04002880237BFF7A2F794B801B7BFF7A2F79C4
:103F14007180137BFF7A2F799E90F956E0FF90F819
:0A3F240035E4F0A3EFF0123E9722FF
:103BCA00182B0000000000000000000000000000A8
:0A3BDA0000000000000000000000E1
:103D590085128385138222860308E6FA08E64A4B10
:103D69002208E6FA08E6F9020596A3E0FEA3E0FFB9
:103D79002290FFFF12059CEFF0C2A922AA06AB0709
:103D890090F957E025E0227C001203C5EF22F8A63E
:103D99000308A60208A60122F8E6FE08E6FFE4FCED
:023DA900FD22F9
:1028DE0090FFFF12059CEBF090FFFE12059CECF0B2
:1028EE00A3EDF0123D7AE58954FCFE123D59E0FB52
:1028FE004EF5899000031205C0E044C0F58B90F9A7
:10290E005BE014605A1470030229B52402600302BE
:10291E002A07123D59123D73EE54FE7009758C163E
:10292E00EEC313EF805F123D59123D73EE54FC70EF
:10293E0010758C2DEF7802CEC313CE13D8F9022961
:10294E00F6123D59123D73D394EAEE9415500B7561
:10295E008CFC7D16123D900229F6AF03022A00125E
:10296E003D59A3E0FEEE700C758C0E123D59A3A3DB
:10297E00E00229F6EE54FE700F758C1D123D59A320
:10298E00E0C313A3E0138060123D59123D73D3943C
:10299E00EFEE9410500A758CFE7D11123D9080481A
:1029AE00123D59E0FF804B123D59A3E0FEEE700B35
:1029BE00758C10123D59A3A3E0802DEE54FE700FBE
:1029CE00758C21123D59A3E0C313A3E01380191295
:1029DE003D59123D73D394EFEE94105010758CFE4A
:1029EE007C007D0F1203C5EF14F58D800C123D593E
:1029FE00E0FF12424D7F00803CAF8C123D59E0FD4E
:102A0E0025E02423F8760008A607AF8DED25E024F7
:102A1E0043F8760008A6077401A805088002C333A0
:102A2E00D8FCF5887410A805088002C333D8FC4280
:0B2A3E0089D2A97F0190000402059CD2
:10424D00123D7A123D59E0FF7410A807088002C391
:0E425D0033D8FCF45289D2A990000102059CCE
:0B436E00EF75F003A4242B123D9722F2
:0B437900EF75F003A42437123D9722DB
:1033B40090F957EFF0FBC2A9E58954FC4BF589AFAE
:1033C4008C784F760008A607AF8DE4FCFDFE784BA1
:1033D400120564EB25E02443123DA1784B120557F6
:1033E400C3EF9BFFEE9AFEED99FDEC98FCC004A997
:1033F40005123D852423123DA1D00012041AC004F5
:10340400C005123D852424F9C3E7785096FF19E7D7
:103414001896FEE4FCFDD001D000EB2FFFEA3EFE3F
:10342400ED39FDEC38FC784B12056490F95BE0143F
:10343400601C14602424027033E47F19FEFDFC78C0
:103444004B12055712041AE47B207A018014784B3E
:1034540012054BE47B0FFA8009784B12054BE47B91
:1034640011FAF9F81204A5784B120564D2A9784D23
:06347400E6FE08E6FF225F
:03000B000232DBE3
:1032DB00C0E0C0F0C083C082C0D075D000C000C0B9
:1032EB0001C002C003C004C005C006C0073088126D
:1032FB00782B123D606005782B123D6A75880102B0
:10330B003399308912782E123D606005782E123D6C
:10331B006A758802023399308A127831123D6060E7
:10332B00057831123D6A758804023399308B117818
:10333B0034123D6060057834123D6A758808804E02
:10334B00308C117837123D6060057837123D6A7505
:10335B008810803A308D11783A123D606005783ACA
:10336B00123D6A7588208026308E11783D123D60A3
:10337B006005783D123D6A7588408012308F0F785A
:10338B0040123D6060057840123D6A758880D00719
:10339B00D006D005D004D003D002D001D000D0D0BD
:0933AB00D082D083D0F0D0E032D2
:08438E00E5FF54077851F62207
:05004E0012438E0022A8
:10426B0012438EE6FF700476098008EFB4010C78D8
:0C427B005176027851E660031680F822AC
:1041E80012438EE6FF7004760C800FEFB401067858
:1041F8005176048005EFB40209227851E66003166F
:0342080080F82219
:10419C0012438EE6FF700476178012EFB401067896
:1041AC005176098008EFB4020C785176027851E60A
:0641BC0060031680F822EA
:103E4A0090F95BE014601314602624027036E5FFD3
:103E5A00540770387851760D802AE5FF54071460AC
:103E6A000904702878517615801A785176038014DF
:103E7A00E5FF54071460090470127851761A800419
:0D3E8A00785176057851E660031680F82225
:103B3E0090F95BE014602714604424027067E5FF7F
:103B4E00540714600D14601024027061785176458C
:103B5E0080537851761B804D785176058047E5FF6E
:103B6E00540714600D146010240270417851765F72
:103B7E00803378517628802D7851760C8027E5FF9A
:103B8E0054071460101460131460162403701E780A
:103B9E0051766D80107851762F800A7851760F808D
:0E3BAE0004E47851F67851E660031680F822A0
:10387500301304D2AED2BE90F95BE0146030146010
:103885005624027079E5FF54071460101460131470
:103895006016240370707851767E80627851763791
:1038A500805C785176138056785176018050E5FF1B
:1038B50054071460101460131460162403704778BD
:1038C5005176A980397851764C80337851761E80AF
:1038D5002D785176078027E5FF5407146010146092
:1038E500131460162403701E785176C08010785129
:1038F5007658800A7851762480047851760A785172
:07390500E660031680F822C2
:102D1700301304D2AED2BE90F95BE0146078147021
:102D270003022E0724026003022E66E5FF5407B450
:102D370007004003022E76902D45F8282873022DB0
:102D47005A022D61022D6B022D75022D7F022D89EE
:102D5700022D9378527603022DF978527601087680
:102D670084022E66785276000876BC022E66785268
:102D77007600087658022E66785276000876260284
:102D87002E667852760008760D022E667852760007
:102D9700087601022E66E5FF5407B40700400302D8
:102DA7002E76902DB0F8282873022DC5022DCF025C
:102DB7002DD9022DE3022DEC022DF5022DFE7852BE
:102DC7007604087607022E66785276010876FD02A9
:102DD7002E66785276000876F9022E6678527600CB
:102DE700087676807A785276000876358071785240
:102DF7007600087615806878527600087604805F3A
:102E0700E5FF5407B407005066902E17F82828737B
:102E1700022E2C022E35022E3E022E44022E4D0289
:102E27002E56022E5F7852760408768980317852C2
:102E3700760208763E802878527601801678527698
:102E47000008768780197852760008763D801078DA
:102E57005276000876198007785276000876067849
:102E670053E61846600908E6161870F31680F02234
:104312007851760A7851E6166005122D1780F5223B
:10432200785176647851E6166005122D1780F522D1
:0C433200AE071FEE600512387580F52202
:0C433E00AE071FEE6005122D1780F5225F
:0C434A00AE071FEE600512431280F52242
:0C435600AE071FEE600512432280F52226
:103BE40046F9120000000000000614000000000066
:013BF40000D0
:10390C0075BC01C390F908E094A890F907E09461A4
:10391C002214FF781AE67814FD08E6FA08E6F58218
:10392C008A8302059A7814860308E6FA08E64A4B5D
:10393C002290F902E0FEA3E0FF90F905E0FCA3E081
:10394C00FDC39FEC9E22F5B7E490F907F0A3F0229B
:10395C00E5BC540690F909F022ED5401C4333354FC
:10396C00C022781C0806E6188606222418F582E484
:10397C0034F9F5832290F907E004F02290F90974E8
:10398C0003F022E490F905F0A3F02290F8FFE0FB9D
:07399C00A3E0FAA3E0F92209
:10406E00EF6019D2BAED6006D2B6D2B78004D2B4E0
:10407E00D2B543BB04E490F919F08017D2B9ED60C4
:10408E0006D2B2D2B38004D2B0D2B143BB02E49016
:06409E00F918F00240D306
:1040D300EF600543BB01800353BBFEEDB4020CEB61
:1040E3005403C454F0FF123965800C1239654480BF
:0B40F300FFEB5403C454F04FF5B7225C
:103FBC0090F945EBF0EF6014D2BAED6006D2B6D2B0
:103FCC00B78004D2B4D2B543BB048012D2B9ED6031
:103FDC0006D2B2D2B38004D2B0D2B143BB0212002B
:0C3FEC002690F945E0F5B3A3E0F5B622FD
:10002600E5BB54FE4FF5BBEDB40208123966442A0F
:10003600F5B12212396544AAF5B175B4FF75B21F40
:0400460043B101229F
:1042D300EF75F003A42412F582E434F9F583EBF0CF
:0742E300A3EAF0A3E9F022B9
:1001EF00EF75F003A42414F8A60308A60208A601CD
:0101FF0022DD
:1027330090F8FDEFF0A3EDF0A3EBF0A3EAF0A3E92B
:10274300F012398FA3F0A3F0A3F090F8FDE0FE128E
:102753003977E060037F012274182E1239797401EE
:10276300F0E5BB54FE4EF5BB75BC0190F904E020C7
:10277300E12E90F8FEE0F5BDE5B754F144021239BD
:1027830052E5BC20E00D1228CA70031239811239B8
:102793000F40EE12390C500512395C800312398850
:1027A30090F909E060030228BB90F8FEE020E00303
:1027B30002283912398F12393D400302288C90F9CF
:1027C30009E0600302288CEF24FFFFEE34FFFEEDE7
:1027D300B50715ECB5061190F904E020E00AE5B75A
:1027E30054F1440AF5B78008E5B754F14406F5B748
:1027F300123954E5BC20E00D1228CA700312398146
:1028030012390F40EE12399790F905E0FEA3E0F577
:10281300828E83E5BF1203A312390C500512395C73
:10282300800312398890F906E004F0700690F905E8
:10283300E004F00227B912398F12393D504B90F959
:1028430009E070451239978D828C83120376F5BEA9
:10285300E5B754F14406123952E5BC20E00D1228C5
:10286300D4700312398112390F40EE12390C50051E
:1028730012395C800312398890F906E004F070067F
:1028830090F905E004F002283C90F904E020E028E8
:10289300E5B754F1440E123952E5BC20E00D12287D
:1028A300D4700312398112390F40EE12390C5005DE
:1028B30012395C800312398890F8FDE0123977E40D
:1028C300F090F909E0FF2212004E90F908E004F0BD
:0B28D3002212004E90F908E004F022F1
:03004B00023A2F47
:103A2F00C0E0C0F0C083C082C0D075D000C000C05D
:103A3F0001C002C003C004C005C006C00790F958FA
:103A4F00E5BBF053BBFEE5B230E11312393160092B
:103A5F0012396E70010612391D75B202802BE5B254
:103A6F0030E310781C7600087600781AA6B575B288
:103A7F00088016E5B230E011123931600912396E43
:103A8F0070010612391D75B20190F958E0F5BBD0DF
:103A9F0007D006D005D004D003D002D001D000D07B
:0A3AAF00D0D082D083D0F0D0E032F6
:030053000235FB78
:1035FB00C0E0C0F0C083C082C0D075D000C000C096
:10360B0001C002C003C004C005C006C00790F95931
:10361B00E5BBF0E5BB54FE4401F5BBE5B230E11E62
:10362B0078171239336012781E1239707001061434
:10363B00FF781BE6781712392475B2028037E5B292
:10364B0030E310781E7600087600781BA6B575B2AD
:10365B00088022E5B230E01D7817123933601378F9
:10366B001E12397070010614FF781BE6FD781712D5
:10367B00392575B20190F959E0F5BBD007D006D0CA
:10368B0005D004D003D002D001D000D0D0D082D04E
:06369B0083D0F0D0E03204
:1040FE00EBF0A3EAF0A3E9F02290F93EE0FBA3E097
:10410E00FAA3E0F92275A102439A03439C03539B41
:09411E00FC227B017AFF7980226A
:1036A10090F92FEEF0A3EFF0A3EDF090F95BE014A9
:1036B100600F146014240270507F007ED07D028060
:1036C1000E7F807EA97D0380067FB07E1E7D047CF7
:1036D10000E5FF5407F9F8120537E47B20FAF9F801
:1036E100123F78C006C00790F92FE0FEA3E0FBAAC5
:1036F10006E4F9F8D007D006123F78C3E49F90F9A9
:1037010033F074049E90F932F0438780759850909D
:10371100F932E0F5BAA3E0F5AA75A101E5A1B4017A
:103721000512411380037595037E007F127D007B96
:10373100017AF879EB12091C90F931E06002D2AC00
:013741002265
:103DAB0090F9341240FEA3ECF0A3EDF0E4FFFE75A6
:103DBB00A101E5A1B401051241138003759503D34D
:103DCB0090F938E09FEE6480F890F937E0648098C2
:103DDB00401E90F93412410A8F828E83120376F5BE
:103DEB0099E59830E1FB5398FD0FBF00010E80CF92
:013DFB0022A5
:1042A30090F95AEFF07B017AF9795A7D017C00127B
:0842B3003DAB90F95AE0FF2237
:103FF80090F9391240FEE4A3F0A3F090F939124188
:104008000AA3E0FEA3E0F5828E83120376FF601315
:104018001242A390F93DE004F070E090F93CE0040E
:0C402800F080D890F93CE0FEA3E0FF22FD
:103E970090F8321240FE90F85D7401F0A374F8F0C8
:103EA700A37435F090F832E0F9A3E0FAA3E090F9B3
:103EB70029C91240FF90F85DE0F9A3E0FAA3E0906A
:103EC700F92CC91240FF124120123F2E1241201235
:0D3ED700000EAC06AD07124120123DAB22DB
:03002300023D0596
:103D0500C0E0C083C082C0D075D000C004C005C06B
:103D150007E59830E02F90F8FBE0FF2401FDE43340
:103D2500FCA3E06D7001EC601974EB2FF582E434AF
:103D3500F8F583E599F090F8FBE004F0E0B41002A3
:103D4500E4F05398FED007D005D004D0D0D082D06F
:043D550083D0E03205
:104127007FFF90F8FCE0FE90F8FBE06E601874EB00
:104137002EF582E434F8F583E0FF90F8FCE004F014
:07414700E0B41002E4F022D5
:103CAF0090F93E1240FEA3ECF0A3EDF0E4FDFCD33F
:103CBF0090F942E09DEC6480F890F941E0648098BF
:103CCF00402F124127EFF460F91241078D828C8348
:103CDF00EF1203A3EFB40A12ED1D70011C1241077E
:103CEF008D828C83E41203A380070DBD00010C802D
:063CFF00BEAE04AF052279
:103BF5004DF8DC000000FF000000000000F0E000D0
:103C050041F8D80041F8D90041F8E90041F8EA0047
:083C150041F8DB0041F8D70083
:103AB900C454F0FEEF4EFFF090F94BE024DCF582A0
:103AC900E434F8F58322E0FF90F94CE022E0FE901F
:103AD900F955E022E090F951FEE033333354F822EE
:103AE90075A101E5A1640122E090F94CFEE0C454FE
:103AF900F0FD22E0FD90F955E0FCED6C22E0FF2499
:103B0900FB24FB22C454F0FD90F8D7E05DFDEE22C2
:103B190090F955E0FFEE6F2290F94CE0540FF0A3B5
:103B2900E0FF22E0FEC454F05FFFEE4FF022F4FE06
:053B3900EF5EF0EE223A
:101DC00090F94CEDF0A3EBF090F94BEFF014604973
:101DD000146079147003021E72147003021E9124A1
:101DE000FA7003021EC4147003021F0B240B60035D
:101DF000021F7290F94DE0FF700790F94CE042FC31
:101E000022EF90F94CB40205E042C88004E0F4529D
:101E1000C890F94CE0F452FC2290F94DE0FF7007B5
:101E200090F94CE042FD22EF90F8D8B40212123A39
:101E3000CFFEEF4EFF90F8D8123AC0E05F42FD228D
:101E4000123ACF90F8D8123B3752FD2290F94DE06C
:101E5000FF700790F94CE042FE22EF90F94CB4027B
:101E600005E042D88004E0F452D890F94CE0F452F6
:101E7000FE2290F94DE07012123AC1C083C0821266
:101E80003ACFFEEF4ED082D083F0123AC1E0F5B0E7
:101E90002290F94DE0FF700790F94CE042F322EFF9
:101EA00090F8D9B40212123ACFFEEF4EFF90F8D953
:101EB000123AC0E05F42F322123ACF90F8D9123BB7
:101EC0003752F322123B217013123AC1C083C082F1
:101ED000123AF1EE4DD082D083F08028EF90F8E9ED
:101EE000B4020E123ACF90F8E9123AB9123B2C80A4
:101EF00013123ACFC454F0F4FEEF5E90F8E9123AB0
:101F0000C0E05EF0123AC1E0F58A2290F94CE0544C
:101F10001CF0A3E0FF7018123AC1C083C082E090A9
:101F2000F94C123AE1FDEE4DD082D083F0803CEFC7
:101F300090F8EAB40220123ACF33333354F8FEEF6C
:101F40004EFF90F8EA123AC0E0FE33333354F85FA4
:101F5000FFEE4FF08015123ACF33333354F8F4FECE
:101F6000EF5E90F8EA123AC0E05EF0123AC1E0F596
:101F7000C122123AE9706E90F94B123B06500724C9
:101F8000FE602C02209B1241C290F94DE0FF7007C9
:101F900090F94CE0429B22EF90F94CB40205E042EC
:101FA0009C8004E0F4529C90F94CE0F4529B229007
:101FB000F94DE0FF700790F94CE0429722EF90F85E
:101FC000DBB40212123ACFFEEF4EFF90F8DB123A6A
:101FD000C0E05F429722123ACFF4FEEF5E90F8DB4A
:101FE000F0EE52972290F94BE0FF24FA6033146030
:101FF000421460612403600302209B90F94DE0FECF
:10200000700790F94CE0429B22EE90F94CB4020527
:10201000E0429C8004E0F4529C90F94CE0F4529B26
:102020002290F94DE090F94C7004E0429422E0F4E3
:1020300052942290F94DE0701574DC2F123AC7C00B
:1020400083C082123ACFFEEF4ED082D083F0123A94
:10205000C1E0F59522123B217013123AC1C083C032
:1020600082123AF1EE4DD082D083F08028EF90F8C2
:10207000D7B4020E123ACF90F8D7123AB9123B2CCD
:102080008013123ACFC454F0F4FEEF5E90F8D712EA
:0C2090003AC0E05EF0123AC1E0F5AD226B
:1041C200EF24FA60111460121460131460142404B2
:1041D2007013E4F5A12275A1012275A1022275A135
:0641E200032275A1042276
:1037DC00AB05AA07EA14601914601B14601D146071
:1037EC001F24FA6020146022240B7023E5805BFFF9
:1037FC0022E5905BFF22E5A05BFF22E5B05BFF2298
:10380C00E5F25BFF22E58A5BFF22E5C15BFF22123A
:10381C003AE97032EA24FB24FB500624FE600C804B
:10382C0047AF021241C2E59A5BFF22E58F5470FA52
:10383C00758F7090F8DAE591F0E4F58FE04591F032
:10384C008A8FE05BFF22EA24FA600F146011146087
:10385C001324037013E59A5BFF22E5935BFF22E5CB
:09386C00955BFF22E5AD5BFF2234
:102A490090F950EFF0A3EDF090F950E0FF123AC57C
:102A5900E04DF0EF14602114603414603B146042BF
:102A690024FA605414607B240B6003022B1290F942
:102A790050123AC4E0F5802290F951E0FF90F8D85D
:102A8900E05F42FD90F950123AC4E0F5902290F9C6
:102A990050123AC4E0F5A02290F950123AC4E0F578
:102AA900B02290F951E0FF90F8D9E05F42F390F934
:102AB90050123AC4E0F5F22290F950E0FF123AC5FB
:102AC900C083C082E090F951123AF590F8E9E05DCF
:102AD900FDEE4DD082D083F074DC2F123AC7E0F5B9
:102AE9008A2290F950E0FF123AC5C083C082123A97
:102AF900DDFD90F8EAE05DFDEE4DD082D083F07403
:102B0900DC2F123AC7E0F5C122123AE9704390F975
:102B190050123B06500724FE6010022BAF1241C22F
:102B290090F950123AC4E0F59A2290F950E0FF1258
:102B39003AC5C083C082123ADDFD90F8DBE05DFD45
:102B4900EE4DD082D083F074DC2F123AC7E0F591B4
:102B59002290F950E0FF24FA601414601B146022DB
:102B69002403704274DC2F123AC7E0F59A2290F9D7
:102B790050123AC4E0F5932290F950123AC4E0F5A4
:102B8900952290F950E0FF123AC5C083C082E0FE59
:102B990090F951E0123B0D4DD082D083F074DC2FB7
:072BA900123AC7E0F5AD226E
:102BB00090F952EFF0A3EDF090F952E0FF123AC510
:102BC000E0FEEDF4FDEE5DF0EF14602114603514CD
:102BD000603C14604324FA6056146077240B600351
:102BE000022C7690F952123AC4E0F5802290F95204
:102BF000123AC4E0F59090F953E0FF90F8D8E05F06
:102C0000F452FD2290F952123AC4E0F5A02290F954
:102C100052123AC4E0F5B02290F952123AC4E0F5EB
:102C2000F290F953E0FF90F8D9E05FF452F322906C
:102C3000F952E0FF123AC5E0FEF58A74DC2F123A31
:102C4000C7C083C08290F953E0C454F0FF90F8E904
:102C5000022D0B90F952E0FF123AC5E0FEF5C17467
:102C6000DC2F123AC7C083C08290F953123AE2FFB8
:102C700090F8EA022D0B123AE9703E90F952123B9D
:102C800006500724FE6010022D161241C290F95220
:102C9000123AC4E0F59A2290F952E0FF123AC5E0E8
:102CA000FEF59174DC2F123AC7C083C08290F953AD
:102CB000123AE2FF90F8DB805290F952E0FF24FADA
:102CC000601414601B1460222403704A74DC2F12F9
:102CD0003AC7E0F59A2290F952123AC4E0F59322ED
:102CE00090F952123AC4E0F5952290F952E0FF12A1
:102CF0003AC5E0FEF5AD74DC2F123AC7C083C0823E
:102D000090F953E0C454F0FF90F8D7E05FF4FFEE81
:072D10005FD082D083F022A6
:10209C0090F955EDF090F954EFF01460441460761B
:1020AC0014700302214314700302216424FA700398
:1020BC000221991470030221EC240B600302223ECE
:1020CC0090F954E0FF123AC5C083C082123AD6FD93
:1020DC00EE6DD082D083F074DC2F123AC7E0F5801D
:1020EC002290F954E0FF123AC5123AD6FDF4FCEEF8
:1020FC005CF59090F8D8E05D62FD74DC2F123AC765
:10210C00C083C082123B19D082D083F090F9541254
:10211C003AC4E0F5902290F954E0FF123AC5C0831E
:10212C00C082123AD6FDEE6DD082D083F074DC2FD3
:10213C00123AC7E0F5A02290F954E0FF123AC5C05C
:10214C0083C082123AD6FDEE6DD082D083F074DC5F
:10215C002F123AC7E0F5B02290F954E0FF123AC5BD
:10216C00123AD6FDF4FCEE5CF5F290F8D9E05D6223
:10217C00F374DC2F123AC7C083C082123B19D08291
:10218C00D083F090F954123AC4E0F5F22290F9544D
:10219C00E0FF123AC5123AD6F4FDEE5DF58A74DC16
:1021AC002F123AC7C083C08290F955E0C454F0FF97
:1021BC0090F8E9E05FFFEE6FD082D083F090F95495
:1021CC00E0FF123AC5C083C082123AD6540FFDEE1E
:1021DC006DD082D083F074DC2F123AC7E0F58A22DE
:1021EC0090F954E0FF123AC5123AD6F4FDEE5DF5C3
:1021FC00C174DC2F123AC7C083C08290F955123AD1
:10220C00E2FF90F8EAE05FFFEE6FD082D083F090AF
:10221C00F954E0FF123AC5C083C082123AD6541C5E
:10222C00FDEE6DD082D083F074DC2F123AC7E0F54E
:10223C00C122123AE9706890F954123B06500724F7
:10224C00FE60270223541241C290F954E0FF123A67
:10225C00C5C083C082123AD6FDEE6DD082D083F019
:10226C0074DC2F123AC7E0F59A2290F954E0FF1271
:10227C003AC5123AD6FDF4FCEE5CF59190F8DBE031
:10228C005D629774DC2F123AC7C083C082123B196F
:10229C00D082D083F090F954123AC4E0F591229098
:1022AC00F954E0FF24FA602B146046146061240397
:1022BC00600302235490F954E0FE123AC5C083C067
:1022CC0082123AFCD082D083F074DC2E123AC7E032
:1022DC00F59A2290F954E0FE123AC5C083C08212DE
:1022EC003AFCD082D083F074DC2E123AC7E0F5931E
:1022FC002290F954E0FE123AC5C083C082123AFC17
:10230C00D082D083F074DC2E123AC7E0F59522749B
:10231C00DC2F123AC7C083C082123AD6123B0D6D25
:10232C00D082D083F074DC2F123AC7C083C082E015
:10233C00FF90F955E0540FFEEF6ED082D083F090F1
:09234C00F954123AC4E0F5AD2287
:0C3C1D00C11241F9470043F948000000C3
:1042870090F948E0FBA3E0FAA3E0F9EA494B229052
:0C429700F948A3E0FAA3E0F5828A832234
:1040340075A101E5A1B4011BEF24FE600C14600E10
:104044002403702375A49C801E75A4DC801975A4B8
:10405400FC801443F580EF24FE6009240270087587
:0A406400A4B8800375A4F8D2BD22B1
:0C43620090F948EBF0A3EAF0A3E9F02288
:10414E0030120CEF70037F862290F947E0FF227544
:10415E00A101E5A1B40107EF04F5A6AFA722EF7008
:07416E0003AFA622AFA72258
:03006B00023C381C
:103C3800C0E0C0F0C083C082C0D075D000C000C052
:103C480001C002C003C004C005C006C007C2127587
:103C5800A101E5A164017019F5A6124287602AE561
:103C6800A530E6047F0180027F00124296ADA7804E
:103C7800151242876013E5A530E6047F0180027FB4
:103C8800001242967D1012059A43A580D007D006EF
:103C9800D005D004D003D002D001D000D0D0D0823B
:073CA800D083D0F0D0E03220
:063C290041F95B01C1132B
:0643A60090F95BEFF0222C
:1042BB00EF6005D213758680E5FFB430037F0122D2
:0842CB0075FF30D2AF7F002225
:08439600301304D2AED2BE22A6
:101AE300444247434D4420537472696E67204275E4
:101AF300666665722046756C6C0D0A002573202599
:101B03005820255820255820255800627573004415
:101B13004247434D44206275733A204275733D300A
:101B23007825302E32582C20506F72743D30782532
:101B3300302E32582C2053706565643D3078253043
:101B43002E32580D0A0063697200444247434D44E4
:101B5300206369723A20436F64653D307825302EE7
:101B630032580D0A0077723100444247434D4420F6
:101B73007772313A2049443D307825302E32582C43
:101B8300205265673D307825302E32582C20446131
:101B930074613D307825302E32580D0A007264315D
:101BA30000444247434D44207264313A2049443D46
:101BB300307825302E32582C205265673D307825F9
:101BC300302E32582C2053697A653D307825302EDB
:101BD30032582C20446174613D20002852656164B1
:101BE300206E756D6265722065786365656420613A
:101BF300206D6178206F6620256420627974657397
:101C030029000D0A002000307825302E32582C2070
:101C13000074623100444247434D44207462313AB8
:101C23002049443D307825302E32582C20526567A8
:101C33003D307825302E32582C204D61736B3D306A
:101C43007825302E32582C20446174613D00307861
:101C530025302E32580D0A00636231004442474357
:101C63004D44206362313A2049443D307825302E7B
:101C730032582C205265673D307825302E32582C4F
:101C8300204D61736B3D307825302E32582C204423
:101C93006174613D0077723200444247434D4420F2
:101CA3007772323A2049443D307825302E32582C11
:101CB300205265673D307825302E34582C204461FE
:101CC30074613D307825302E32580D0A007264322B
:101CD30000444247434D44207264323A2049443D14
:101CE300307825302E32582C205265673D307825C8
:101CF300302E34582C2053697A653D307825302EA8
:101D030032582C20446174613D00746232004442B5
:101D130047434D44207462323A2049443D3078258C
:101D2300302E32582C205265673D307825302E34C2
:101D3300582C204D61736B3D307825302E32582C52
:101D430020446174613D0063623200444247434D65
:101D530044206362323A2049443D307825302E32A4
:101D6300582C205265673D307825302E34582C206E
:101D73004D61736B3D307825302E32582C204461F1
:101D830074613D004552524F523A204949432066FF
:101D930061696C65642025642C204949434164646E
:101DA300723D307825302E32582C205265674164BD
:0D1DB30064723D307825302E32580D0A0044
:083C2F0041F8D20041F8D00079
:10006E00A3F090F8B7E0FF90F8BAE0FCA3E090F9A7
:10007E0020FD7B017AF879BEE4F0A304F02278BE6D
:10008E007CF87D017BFF120755EF227BFF7A1C79EE
:10009E000A90F8D4E024BEF582E434F8F583E0FF4C
:1000AE00E490F835F0A3EFF02290F922E090F924D5
:1000BE00FDE0FBA3E0FAA3E0F9A3E0FFA3E090F9D3
:1000CE0002CFF0A3EFF02278BE7CF87D017BFF1209
:1000DE000755EF2278BE7CF87D017BFF120755EFA6
:1000EE002290F8BEF090F8B7E0FF90F8B9E07AF8F9
:1000FE0079BE90F927FD7B01E4F0A32278BE7CF84F
:10010E007D017BFF120755EF2290F8B9E0FEA3E0C8
:10011E004EF0A3E0F022F0A3EDF0A3EBF0A3EAF093
:10012E00A3E9F090F8D3E4F0A3740AF0E4A3F0A3EB
:10013E00F022A3F0A37401F0A322E0FEA3E0FF904F
:10014E00F8D3E0FCA3E0FDC39FEC9E22E0FFE49019
:10015E00F837F0A3EFF022E0FFA3E0CF90F839F0EC
:10016E00A3EFF022E0FD7B017AF879BEA3E0FFA3B6
:10017E00E022D390F8D4E0940090F8D3E0940022DB
:10018E00C390F8D6E0940390F8D5E094002278BEA0
:10019E007CF87D017BFF120755EF22A3E024FDF0D2
:1001AE0090F8D3E034FFF02290F8B7E0FF90F8B962
:1001BE00E0227BFF90F8B6E0FFA3E0227BFF7A1CE3
:1001CE0079052290F8BEE0FF90F8BBE02290F8BED1
:1001DE00E0FF90F8BDE0227BFF7A1C795190F8BECB
:0101EE0022EE
:100FFC0012412790F95CEFF0F4700302132BE0FF21
:10100C0090F8D2E0FE04F074BE2EF582E434F8F5CC
:10101C0083EFF090F8D2E0D39412400E7BFF7A1A53
:10102C0079E3123E97E490F8D2F090F95CE0FF641B
:10103C000A6008EF640D600302132BE490F8D2F001
:10104C0090F86374FFF0A3741AF074FF12014074EB
:10105C00FFF0748012014074F8F0A374B6120141D1
:10106C0074F8F0A374B812014174F8F0A374BA12B6
:10107C00014174F8F0A374BCF07B017AF879BE12CC
:10108C00184AE490F8C1F07A1B790E12008C701E8D
:10109C007A1B79121213311201B6FD90F8BBE0FBEA
:1010AC0012406E90F8B7E090F8D0F002132B7A1B38
:1010BC00794912008C703F7A1B794D1201C0CF1206
:1010CC0000AF123E97D21290F8B7E090F947F0902B
:1010DC00F948E0FBA3E0FAA3E0F9EA494B700302FC
:1010EC00132B90F948A3A3E0F5828A837D10E4FFCB
:1010FC0012059A02132B7A1B79681200D5701E7A8E
:10110C001B796C12133190F8BBE090F8BEF0120111
:10111C00B690F92712007F12353E02132B7A1B79F9
:10112C00A01200D560030211C37A1B79A41201C06E
:10113C0090F835CFF0A3EFF090F8B8E0FFA3E0CF34
:10114C0012015D90F8BA120165123E97D390F8BB6C
:10115C00E0941290F8BAE09400400312143490F822
:10116C00B7E04401FFC00790F8B912017290F9275B
:10117C00CFF0A3EFF0D00712353EEF600302132B34
:10118C0090F8D3F0A3F090F8BA1201485026ED5421
:10119C000F70061201CA123E9790F8D4E0540770F3
:1011AC000312144812009912145270DA90F8D3E01A
:1011BC0004F080D20212C27A1C79141200E2702759
:1011CC007A1C79181213E712353EEF600302132BC9
:1011DC001201D1FEEF6E1200EF04F012353EEF60FB
:1011EC000302132B0212F07A1C795B1200E27028B6
:1011FC007A1C795F1213E712353EEF600302132B52
:10120C001201D1F4FEEF5E1200EF04F012353EEF46
:10121C00600302132B0212F07A1C799812010A70E7
:10122C00171201177A1C799C12136490F8BDE01206
:10123C00006E12347A02132B7A1C79D012010A70C8
:10124C007B1201177A1C79D4121364D390F8BDE089
:10125C00941290F8BCE09400400312143490F8B748
:10126C00E04401FFC00790F8BAE0FCA312017290B1
:10127C00F920CFF0A3EFF0D00712347AEF6003021D
:10128C00132B90F8D3F0A3F090F8BC120148502621
:10129C00ED540F70061201CA123E9790F8D4E05428
:1012AC0007700312144812009912145270DA90F855
:1012BC00D3E004F080D21201CA0213287A1D790DF2
:1012CC0012019C70281201177A1D791112139712B2
:1012DC00347AEF704A1201DBFEEF6E12006E12349C
:1012EC007AEF703B1201E51200AC0213287A1D79DB
:1012FC004A12019C70291201177A1D794E1213970C
:10130C0012347AEF70191201DBF4FEEF5E12006EEC
:10131C0012347AEF70091201E51200AC123E97906C
:10132C00F95CE0FF227BFF90F8B6E0FFA3E090F8B9
:10133C0035CFF0A3EFF090F8B8E0FFA3E090F837CA
:10134C00CFF0A3EFF090F8BAE0FFA3E090F839CF1C
:10135C00F0A3EFF0123E97227BFF90F8B6E0FFA3CC
:10136C00E090F835CFF0A3EFF090F8BAE0FFA3E0EF
:10137C0090F837CFF0A3EFF090F8BCE0FFA3E0902B
:10138C00F839CFF0A3EFF0123E97227BFF90F8B61E
:10139C00E0FFA3E090F835CFF0A3EFF090F8BAE0BF
:1013AC00FFA3E090F837CFF0A3EFF090F8BCE0FF8C
:1013BC00A3E090F839CFF0A3EFF0123E9790F8B776
:1013CC00E04401FF90F8BAE0FCA3E0FD7B017AF861
:1013DC0079BE90F920E4F0A304F0227BFF90F8B6DC
:1013EC00E0FFA3E090F835CFF0A3EFF090F8B8E071
:1013FC00FFA3E090F837CFF0A3EFF090F8BAE0FF3E
:10140C00A3E090F839CFF0A3EFF0123E9790F8B725
:10141C00E04401FF90F8B9E0FD7B017AF879BE90C9
:10142C00F927E4F0A304F022E4F0A37412F07BFF9C
:10143C007A1B79DE90F835F0123E97227BFF7A1CEE
:10144C007908123E9722123E9790F8D4E004F022CD
:10353E0090F922EF12012490F922E0FE90F8D0309B
:10354E00E01AE0FFEE147AF9792390F902120103E2
:10355E001235ECC0061200B7E4A3801EE0FF90F90E
:10356E0022E0FD7B017AF9792390F902E4F0A312AF
:10357E0035ECC0061200B7A37402F090F8D0E0FF4D
:10358E00122733D0E04F90F8D1F090F8D1E06026BA
:10359E0090F8D3E0FEA3E0FF12433E1201804003F9
:1035AE001201A990F8D6E004F0700690F8D5E00468
:1035BE00F012018E408190F8D1E0FF601B7BFF7A04
:1035CE001D79871200AE90F92212015A90F923E06C
:1035DE00FFE412016A123E9790F8D1E0FF2204F048
:0D35EE00A3F012273390F8D1EFF0E0FE2299
:10347A0090F91AEFF0A3EC12012490F91AE0FE90E9
:10348A00F8D030E017E0FFEE14123520C00690F9AC
:10349A001AE090F91D1200BEE4A38019E0FF90F92A
:1034AA001AE0123520C00690F91AE0FD90F91D12B3
:1034BA0000BFA37402F090F8D0E0FF122733D0E0E7
:1034CA004F90F8D1F090F8D1E0602690F8D3E0FE62
:1034DA00A3E0FF12433E12018040031201A990F8B3
:1034EA00D6E004F0700690F8D5E004F012018E40A0
:1034FA008990F8D1E0FF60187BFF7A1D7987120066
:10350A00AE90F91A12015A90F91B120165123E97F0
:10351A0090F8D1E0FF22FD7B017AF9791B90F9023C
:10352A00E4F0A37402F0A314F012273390F8D1EF59
:04353A00F0E0FE229D
:030000000239A31F
:0C39A300787FE4F6D8FD7581530239EA04
:10028000E709F608DFFA8046E709F208DFFA803E60
:1002900088828C83E709F0A3DFFA8032E309F6084D
:1002A000DFFA8078E309F208DFFA807088828C83B5
:1002B000E309F0A3DFFA806489828A83E0A3F60869
:1002C000DFFA805889828A83E0A3F208DFFA804C43
:1002D00080D280FA80C680D4806980F2803380101A
:1002E00080A680EA809A80A880DA80E280CA803383
:1002F00089828A83ECFAE493A3C8C582C8CCC583FB
:10030000CCF0A3C8C582C8CCC583CCDFE9DEE780CA
:100310000D89828A83E493A3F608DFF9ECFAA9F049
:10032000EDFB2289828A83ECFAE0A3C8C582C8CC9F
:10033000C583CCF0A3C8C582C8CCC583CCDFEADEB8
:10034000E880DB89828A83E493A3F208DFF980CC1A
:1003500088F0EF60010E4E60C388F0ED2402B40413
:100360000050B9F582EB2402B4040050AF232345BA
:0603700082239002D0730D
:10037600BB010CE58229F582E5833AF583E022503C
:1003860006E92582F8E622BBFE06E92582F8E22286
:0D039600E58229F582E5833AF583E49322A0
:1003A300F8BB010DE58229F582E5833AF583E8F090
:1003B300225006E92582C8F622BBFE05E92582C83C
:0203C300F22224
:1003C500BC000BBE0029EF8DF084FFADF022E4CC1C
:1003D500F875F008EF2FFFEE33FEEC33FCEE9DECE5
:1003E500984005FCEE9DFE0FD5F0E9E4CEFD22ED2B
:1003F500F8F5F0EE8420D21CFEADF075F008EF2F75
:10040500FFED33FD4007985006D5F0F222C398FD65
:050415000FD5F0EA2202
:10041A00E88FF0A4CC8BF0A42CFCE98EF0A42CFC81
:10042A008AF0EDA42CFCEA8EF0A4CDA8F08BF0A4FF
:10043A002DCC3825F0FDE98FF0A42CCD35F0FCEB5E
:10044A008EF0A4FEA9F0EB8FF0A4CFC5F02ECD3923
:0F045A00FEE43CFCEAA42DCE35F0FDE43CFC2290
:1004690075F008758200EF2FFFEE33FECD33CDCC4A
:1004790033CCC58233C5829BED9AEC99E5829840CD
:100489000CF582EE9BFEED9AFDEC99FC0FD5F0D6AA
:10049900E4CEFBE4CDFAE4CCF9A88222B800C1B9D4
:1004A9000059BA002DEC8BF084CFCECDFCE5F0CB12
:1004B900F97818EF2FFFEE33FEED33FDEC33FCEB4B
:1004C90033FB10D703994004EB99FB0FD8E5E4F906
:1004D900FA227818EF2FFFEE33FEED33FDEC33FCF3
:1004E900C933C910D7059BE99A4007EC9BFCE99AE7
:1004F900F90FD8E0E4C9FAE4CCFB2275F010EF2F2C
:10050900FFEE33FEED33FDCC33CCC833C810D7072B
:100519009BEC9AE899400AED9BFDEC9AFCE899F866
:0E0529000FD5F0DAE4CDFBE4CCFAE4C8F922F9
:103F7800C2D5E830E70FB2D5E4C39BFBE49AFAE474
:103F880099F9E498F8EC30E717B2D5123FAE12046D
:103F9800A5E4C39BFBE49AFAE499F9E498F8800352
:103FA8001204A530D50DE4C39FFFE49EFEE49DFDF9
:043FB800E49CFC2267
:10053700E86010ECA2E713FCED13FDEE13FEEF13DA
:04054700FFD8F022C7
:0C054B00E6FC08E6FD08E6FE08E6FF22DC
:0D055700E6FB08E6F908E6FA08E6CBF82214
:0C056400ECF608EDF608EEF608EFF622C3
:10057000D083D082F8E4937012740193700DA3A31A
:1005800093F8740193F5828883E47374029368602E
:06059000EFA3A3A380DF2E
:060596008A838982E473F0
:10059C00E5132582F582E5123583F583B5120485C2
:1005AC0082132210AF06858213F51222858213F571
:0405BC0012D2AF2286
:0D05C000E5132582F582E5123583F58322CF
:1017C100E508300C0104F823282463F582E434F899
:1017D100F5832290F860300C0390F863E475F00112
:1017E1001209C302094860EAC50C7002150B14C541
:1017F1000C200C04FF02439E90F86074FFF5F00288
:1018010009DAFF0242FEE5096006D509037F0022DD
:10181100200C0F1242EAEF6008050CE50C7002057E
:101821000B2290F8601209BA120948FF60E890F89B
:1018310060E475F0011209C380DC121811EFC0E0F9
:10184100121803D0E040F3809DD20C8002C20C90AC
:10185100F8601209F1E4F50AF508F50BF50C7509C4
:1018610000C20BC209C20AC20D1217D4FF7005AF24
:101871000A7E0022B425301217D4FF24D0B40A0006
:10188100500C75F00AC509A42509F50980E924CF92
:10189100B41A00EF5002C2E5021AAFD20A80D8D2C0
:1018A1000980D4D20D80D0EF121803500812183BD2
:1018B100EF600E80A9EFC0E0121811D0E06F609EBA
:1018C100EF60741217E780A7121811EF6069E5093C
:1018D100700705098003121811EF6014200D0E1214
:1018E10017C1E475F0011209C3EF120961D509E6C8
:1018F100200D040508050A80BA121807EFC0E0128E
:101901001803D0E050041217E7E4FF200D0E121760
:10191100C1E475F0011209C3EF120961EF70DA2019
:101921000D040508050A808BE509600205091218F6
:101931003B121807EF70C6300C04E41217E7E50AF2
:1019410060030218707EFF7FFF22200D1174FFFCDF
:10195100FDFEFF1217C11209BA1209A005080218EB
:101961005FD0E080D27900800A7910800679088002
:1019710002790AD20EE50960020509E9C0E01218F0
:101981003BEF60DD121811BF2D04D20B8003BF2B7A
:101991000912183BEF60CA121807D0E0B40A02809E
:1019A10033B40802802EBF302770027408C20EC003
:1019B100E0121807D0E0BF78028003BF581605096E
:1019C100D509028007D50904D20E800B7410801945
:1019D1007002740ABF000AEFF8E4FCFDFEFF021A70
:1019E10062C0E0EF1217E7D0E0F9E4FCFDFEFFE989
:1019F100C0E0ECC0E0EDC0E0EEC0E0EFC0E01218E6
:101A010007EFF8D0E0FFD0E0FED0E0FDD0E0FCD061
:101A1100F0E8604DB461004007B47B005002C2E5BC
:101A210024D0503DFA24F6500724F95034240AFA00
:101A3100EAB5F000502BCFA9F0A42FFF92D5E9C54C
:101A4100F0CEA4A2D53EFE92D5E9C5F0CDA4A2D593
:101A51003DFD92D5E9C5F0CCA4A2D53CFCC20E80D7
:061A61008EE8C0E0200D3C
:101A67002A200E08050A300B031209921217C11219
:101A770009BA050820090B200A0DEE8FF012097329
:101A870080091209A08004EF120961D0E01217E75C
:101A970002185F200D101217C11209BA0508E50BCD
:101AA700850CF012097380E8120570192953196A19
:101AB7005818A04C189C42187848196E4F19724450
:101AC70018C943196649197255194B46194B4519D7
:0C1AD7004B4718A42A1A9A4E000018A8C9
:1005CD00E3F5F009E208B5F06D606B80F3E3F5F04B
:1005DD0009E608B5F060605E80F387F009E608B5BE
:1005ED00F054605280F487F009E208B5F048604697
:1005FD0080F488828C8387F009E0A3B5F0386036EB
:10060D0080F488828C8387F009E493A3B5F027608A
:10061D002580F388828C83E3F5F009E0A3B5F0160D
:10062D00601480F388828C83E3F5F009E493A3B51D
:10063D00F004600280F20206F8808580E7808E80EB
:10064D00D2803C8015806C807E809B80B5808B80B5
:10065D00A1804F8070803A02070E89828A83ECFA5E
:10066D00E493F5F0A3C8C582C8CCC583CCE493A3AD
:10067D00C8C582C8CCC583CCB5F070606E80E189E9
:10068D00828A83E493F5F0A3E208B5F05E605C80A6
:10069D00F289828A83E0F5F0A3E608B5F04D604B50
:1006AD0080F389828A83E0F5F0A3E208B5F03C601F
:1006BD003A80F389828A83E493F5F0A3E608B5F0D6
:1006CD002A602880F2805D89828A83ECFAE493F5B2
:1006DD00F0A3C8C582C8CCC583CCE0A3C8C582C869
:1006ED00CCC583CCB5F004600280E27F00F845F004
:1006FD00600EE863F0806480D395F01F40027F01A7
:10070D002289828A83ECFAE0F5F0A3C8C582C8CCB1
:10071D00C583CCE0A3C8C582C8CCC583CCB5F0CB0E
:10072D0060C980E389828A83ECFAE0F5F0A3C8C53D
:10073D0082C8CCC583CCE493A3C8C582C8CCC5837D
:10074D00CCB5F0A760A580E288F0ED2402B40400DA
:10075D005099F582EB2402B40400508F2323458277
:05076D00239006467315
:10000E00E4FFFE120948600C0FEF70010E09E97053
:05001E00F20A80EF2250
:10077200E3F5F009E208B5F06BDFF58067E3F5F029
:1007820009E608B5F05EDFF5805A87F009E608B59C
:10079200F052DFF6804E87F009E208B5F046DFF648
:1007A200804288828C8387F009E0A3B5F036DFF6B9
:1007B200803288828C8387F009E493A3B5F025DF29
:1007C200F5802188828C83E3F5F009E0A3B5F0146B
:1007D200DFF5801088828C83E3F5F009E493A3B5FA
:1007E200F002DFF40208A1808780E9809080D48043
:1007F2003E8015806E807E809D80B7808D80A38034
:10080200518074803C0208AD89828A83ECFAE493B9
:10081200F5F0A3C8C582C8CCC583CCE493A3C8C5F0
:1008220082C8CCC583CCB5F076DFE3DEE180708987
:10083200828A83E493F5F0A3E208B5F062DFF480E4
:100842005E89828A83E0F5F0A3E608B5F051DFF510
:10085200804D89828A83E0F5F0A3E208B5F040DF9B
:10086200F5803C89828A83E493F5F0A3E608B5F02B
:100872002EDFF4802A8002805789828A83ECFAE490
:1008820093F5F0A3C8C582C8CCC583CCE0A3C8C584
:1008920082C8CCC583CCB5F006DFE4DEE280007FFF
:1008A200FFB5F0020F2240027F012289828A83EC87
:1008B200FAE0F5F0A3C8C582C8CCC583CCE0A3C8D2
:1008C200C582C8CCC583CCB5F0D5DFE5DEE380CFE9
:1008D20089828A83ECFAE0F5F0A3C8C582C8CCC548
:1008E20083CCE493A3C8C582C8CCC583CCB5F0AF92
:1008F200DFE4DEE280A988F0EF60010E4E60ABED2E
:100902002402B404005098F582EB2402B40400508F
:0A0912008E23234582239007E9732A
:10091C00EF4E6012EF60010EEDBB010B89828A83F2
:10092C00F0A3DFFCDEFA2289F05007F709DFFCA9FF
:0C093C00F022BBFEFCF309DFFCA9F02256
:103F2E0090F929E0FFA3E0FEA3E0CF90F891F0A373
:103F3E00EEF0A3EFF090F92CE0CBF0A3E0CAF0A3E3
:103F4E00E0C9F07F2290F894AD82AC831209488DBF
:103F5E00828C83F0A309E970010ADFEC90F92CE062
:0A3F6E00FBA3E0FAA3E0F90214C17E
:1039AF00020A12E493A3F8E493A34003F68001F212
:1039BF0008DFF48029E493A3F85407240CC8C33319
:1039CF00C4540F4420C8834004F456800146F6DFE8
:1039DF00E4800B0102040810204080903BBCE47E81
:1039EF00019360BCA3FF543F30E509541FFEE493DD
:1039FF00A360010ECF54C025E060A840B8E493A3A4
:103A0F00FAE493A3F8E493A3C8C582C8CAC583CACE
:103A1F00F0A3C8C582C8CAC583CADFE9DEE780BE86
:013C3700008C
:10094800BB010689828A83E0225002E722BBFE02AD
:09095800E32289828A83E49322E0
:10096100BB010689828A83F0225002F722BBFE0175
:02097100F3226F
:10097300BB010A89828A83F0E5F0A3F0225006F7CF
:0F09830009A7F01922BBFE06F3E5F009F31922CC
:0E099200C3E49FFFE49EFEE49DFDE49CFC2276
:1009A000BB010789828A830209FA5005E9F802052A
:0A09B00064BBFE05E9F8020A062206
:0909BA00E0FBA3E0FAA3E0F9223E
:1009C300F8E0FBA3A3E0F925F0F0E58215827002BD
:0709D3001583E0FA38F02261
:1009DA00F8E0FBA3A3E025F0F9F0E58215827002A6
:0709EA001583E038FAF0224A
:0909F100EBF0A3EAF0A3E9F02207
:10145C00E50D2491F582E434F8F583E0050D229036
:10146C00F88E30070390F891E475F0011209C3026D
:10147C0009482000E97F2ED2008018EF540F2490E9
:10148C00D43440D4FF30040BEF24BFB41A00500303
:10149C002461FFE50E6002150E0511E511700205C1
:1014AC001030070E90F88EE475F0011209C3EF02AC
:1014BC0009610241757403D2078003E4C207F50D7C
:1014CC0090F88E1209F1E4F50EF510F511E50E60A9
:1014DC00077F2012149F80F5750FFFC201C200C256
:1014EC0002C203C205C206C20812146BFF700D3093
:1014FC0007057F001214B0AF11AE1022B4255FC2E5
:10150C00D5C20412146BFF24D0B40A00501A75F023
:10151C000A780E30D50508B6FF0106C6A426F620BB
:10152C00D5047002D20380D924CFB41A00EF500432
:10153C00C2E5D2040216B1D20180C6D20080C0D25C
:10154C000280BCD2D580BAD20580B47F2012149F01
:10155C002002077401B50E0040F112145CFF121446
:10156C009F0214D9D208D206809512145CFB121477
:10157C005CFA12145CF94A4B700679827A177BFF7D
:10158C0020022EE50E602A7E008E827583001203E7
:10159C007660060EEE650F70F0C2D5EBC0E0EAC0C7
:1015AC00E0E9C0E0EE1216F8D0E0F9D0E0FAD0E0B5
:1015BC00FB120948FF60AAEBC0E0EAC0E0E9C0E01A
:1015CC0012149FD0E02401F9D0E03400FAD0E0FBF3
:1015DC00E50F0460DCD50FD980877BFF7A1679F490
:1015EC00D202809C791080027908C206C208800859
:1015FC00D2D5790A8004790AC2D5E50F047002F5B8
:10160C000FE4FAFDFEFF12145CFC7B0820011312A0
:10161C00145CFD7B1030000A12145CFE12145CFF8B
:10162C007B20EC3382D592D55013C3E43000069F57
:10163C00FFE49EFEE42001039DFDE49CFCE4CBF85A
:10164C00C201EC700CCFCECDCCE824F8F870F3804E
:10165C0017C3EF33FFEE33FEED33FDEC33FCEB330E
:10166C00FB994002FB0FD8E9EB300105F8D0E0C440
:10167C0048B201C0E00AEC4D4E4F78207B0070C29E
:10168C00EAB50F0040BCC0E01216FAD0F0D0E02052
:10169C000104C4C0E0C4B201C0F0121488D0F0D56B
:1016AC00F0EB0214D912057015765315F058154746
:1016BC004C15434215F44F15FC4415FC49155C437D
:0816CC0016025515E64615E66D
:1016D4004515E64717A250154B2D154F2E15722BA5
:1016E400155323157020178B2A150B480000156A13
:1016F4003F3F3F00790AA2D5200314300509B910F1
:10170400020404B9080104A2D520060250010420F1
:1017140002689202B50E005034C0E07F20300319F5
:101724007F30A20272067205500F121751C202C214
:1017340006C205C2087F30800F300503E9C0E012FD
:10174400149F300503D0E0F9D0E0B50ECC30051776
:101754007F30B9100C12149F7F583004077F7880B3
:1017640003B9080312149F3002057F2D02149F7FD2
:10177400202008F87F2B2006F322920280CF286EC7
:10178400756C6C2900D20112145C3001F8C2017826
:101794000E30D50108F602150B2D5043495812148A
:1017A4005C2403B405004001E490179D9312149047
:0D17B400743A121490D203750E040215F061
:1042EA0010140B124384BF0D027F0A02417590F924
:0442FA005DE0FF2262
:08439E0090F95DEFF0D214224A
:1042FE00EFC394094005EF940E4004EFB42003D3AE
:04430E008001C32245
:0C09FA00ECF0A3EDF0A3EEF0A3EFF02270
:0C0A0600ECF208EDF208EEF208EFF2222C
:10417500EFB40A07740D124180740A309811A8999A
:10418500B8130CC2983098FDA899C298B811F630AA
:0741950099FDC299F5992282
:0A4384003098FDAF99C2987E002228
:00000001FF
